:100000008A01B501B6014729DB2870088207012A59
:10001000012A452D0E281F283028392EC71F862279
:10002000471F012A47137108053C031C012A710868
:100030008207012AB62DC02DC22DCC2DCE2DC71F73
:100040008622471F012A47137108053C031C012A19
:1000500071088207012A012A012AD82DE22DE42DF8
:10006000C71F8622471F012A471371080E3C031C35
:10007000012A71088207012A012A012AF72D012E7F
:10008000032E052E072E0C2E1C2E012A1E2E282E86
:100090002A2E342E74088207442C4A2C622C6B2C96
:1000A000742C9A2C9A2C9A2C9A2C9A2C9A2C9A2C46
:1000B0009A2CA22C74088207442CAE2CAE2CAE2CA9
:1000C000E12CE12CE12CE12CE12CE12CE12CE12CC8
:1000D000E12CE12C1A08FC001819D5289818D5280D
:1000E0000F23270803197B28280803197B28F00110
:1000F000F101E70108007008820784288C28912804
:1001000091289128912891286708031D9A287C0836
:10011000243C0319B6289A286708063C0319BB2813
:100120009A287C082C3C0319BF287C082A3C031918
:10013000BF289A287C08083C031DA728E708031954
:10014000B528E70320300F2308300F23B5286708B0
:10015000A03E84007C08800087110A3C0319C9284E
:1001600067081F3C031CC928E70A08000130F0009B
:10017000F101E701A7280230F000E7010800F10AC9
:100180006708A03E84007C088000E70147178711BC
:1001900008008715E701F1014713F008031DD32874
:1001A0000630F0000800F0010800E701F0014713F5
:1001B000181218160800FE00030E8301FF00040841
:1001C000FD000B1184308100EF202B218C1A6A2056
:1001D0007D0884007F0E8300FE0E7E0E0900A30DB5
:1001E00020081502A0002108031C210A1602A10004
:1001F00006302102F13003192002031802290029D8
:100200002310032923141508A0001608A100A40B2D
:100210001D290A30A400C9010830CA00A30D031823
:10022000C90ACA0B0E29A30DA50D053049020318F2
:100230001B2925141C292510A60A0F302302031D93
:1002400008000530240203192A29031C2929A403C4
:100250000800A40A0800AF03031D3429C60A6E086B
:100260004602031D3429C601B10D07183929311082
:100270003A293114A20D071A3F29221040292214CD
:10028000BE0D051A45293E1046293E140800E70117
:10029000A601B701C501BF01C001C101C201C3016F
:1002A000C401C701F001F101F4013E14311422141C
:1002B000C6010230EE0003178F0103130A30A400B9
:1002C0001E308500860187018316D33081000630F9
:1002D0009F0085010516860187010714071507167B
:1002E0008716871783120730970010148316033080
:1002F000920083120F309D0001309B00121583166F
:100300001930990098168312181398171816362268
:1003100060308B0097302B22AE01A701A801A90104
:10032000C710FD21783C031D8C29F408031D8C297E
:10033000F121333C031D8C29F121783C031D8C29CC
:10034000B50192227A22C71396302B222908AA00DF
:100350002808A9008711F121A8008715F121A7001D
:10036000783C0319A6292E08A13E2B224719A7176E
:100370002708F926D200A7134719AA172A08F92631
:10038000AC00AA13D2080319D229AC080319D92941
:1003900052082C020319CD29E529AE080319D929E1
:1003A000AE03D9292A08A7002C08D200D2080319C5
:1003B000E52952084C3C031DDF294711E829520862
:1003C000463C031DE7294715E829AE0AE82915230D
:1003D0002A08783C03198A292E08063C031DA62901
:1003E0008A298B1700008B132608063C0318F12975
:1003F000A60125087F398B1708008B172724F224C4
:1004000005288B13A6080319FD29A60125087F39A5
:100410008B170800871A08008316FF3086008312A6
:100420008516851585100511060805150339033C49
:10043000031D122A85148511831686018312080074
:10044000871A0800B8000A2238088600851185122C
:10045000051105150800871A0800B8000A22380897
:100460008600851585120511051508003D304D26BD
:1004700036304D260514A52268227A22922268225F
:100480009222283020220030202241302B2280303E
:100490002B22A1302B223530202236302022213051
:1004A0002B225230922565309225763092253130BC
:1004B00092252E3092253330922592220800283042
:1004C000B20000302022C0302B22B20B612A08007B
:1004D0004030B2000230B30000302022C0302B2266
:1004E000B20B6C2AB30B6C2A08002830C107031C1E
:1004F0007A2AC20A4108C30020224208C4002022EE
:1005000040302B2236083702C5000800A0302022D8
:100510001E30202240302B2208002830BF07031C49
:10052000922AC00A3F0820224008202224302B2291
:1005300008002830E807031C9E2AE90A68082022E0
:100540006908202224302B220800A030E8001E3049
:10055000E9009E2AAB0036083702C5002B08443C50
:100560000319D22AC71CBB2AC7102B08203C031929
:10057000BB2AF523C22AB508031DC22A2B08203C3A
:100580000319E32AB50A20302B022022C0302B2287
:100590003508273C0318E32AC714B501B60AB70A81
:1005A0008D22DA2AB5080319E32AC710B501B60A65
:1005B000B70A8D223708C33C031CF22A3608073CD1
:1005C000031CEB2AE42AC710350820223608202213
:1005D00021302B2208000730B600C50A75225F22A1
:1005E0009222E42AB601B501C101C201C301C401CE
:1005F000BF01C001B701C5017A229222682292226E
:100600004714E32A53080A3C031D082B2030D3006B
:1006100053080D3C031D0E2B2030D3000800831619
:10062000981C102B8312990008005208413C0319B2
:10063000F42B5208423C0319F42B1430B2006530FD
:1006400084000008840A800084038403B20B212BF9
:100650005B087A3C031DCF2B5A08633C031DCF2B4C
:1006600059087A3C031DCF2B5808633C031DCF2B40
:100670005708203C031DCF2B2630F300ED262A3CE3
:100680000319522B720856020319522B2730F3001C
:10069000ED2656020319522B2830F300ED265602A0
:1006A000031DCE2B653055020319BA2B623055025B
:1006B0000319BA2B643055020319BA2B2930F30001
:1006C000ED26793C031D682B613055020319BA2BC6
:1006D0002A30F300ED26793C031D722B633055025E
:1006E0000319BA2BF30AED26793C031D7B2B6630E8
:1006F00055020319BA2BF30AED26793C031D842B0E
:10070000673055020319BA2BF30AED26793C031D15
:100710008D2B683055020319BA2BF30AED26793C6C
:10072000031D962B693055020319BA2BF30AED26E7
:10073000793C031D9F2B6A3055020319BA2BF30A2B
:10074000ED26793C031DA82B6B3055020319BA2BFB
:10075000F30AED26793C031DB12B6C3055020319C9
:10076000BA2BF30AED26793C031DCE2B7A305502C5
:10077000031DCE2BC719CF2BC7154430AA22093031
:10078000B2005B30840000080F2302230008AA2275
:100790008403B20BC32B4430AA220800C7115608A9
:1007A0006E3C031DED2B55086E3C031DED2B5408CC
:1007B0006E3C031DED2B53086E3C031DED2BC71D36
:1007C000080053080F230D300F230A300F2353085E
:1007D000AA224430AA22C7110800C71DF42B5308CF
:1007E0000F2302235308AA2208005408203C0319AF
:1007F0000800B50A1230B200553084000008203CD1
:100800000319082CB50A840AB20BFE2BB5010800A7
:100810003508B200B20A00302022C2302B22B20BBF
:100820000B2C92225330350784003508B20020305B
:1008300000022022C0302B228403B20B172C0800A8
:100840006C0820226D08202221302B220800BE08CF
:10085000031D3C2CC608031D442CC60AF40A87114C
:100860000430EE0074080E3C0319372C4A28A522E8
:100870006822F4017A22E4223E0831052205031998
:10088000442CE7080319871508005330922554308B
:100890009225080097302B22A1302B220430EC0047
:1008A000ED0120242630EB00A52268229E2286221C
:1008B0004524313092253A3092256B08F300ED261D
:1008C000A924442CED0A20242730EB00992245244A
:1008D000323092255B2CED0A20242830EB0099223F
:1008E0004524333092255B2CEC01ED0AED0A2024DF
:1008F0009922413092254330922546309225473047
:10090000922548309225493092254A3092254B3025
:1009100092254C3092255A30922599222930EB00AD
:10092000F3000A30B200ED269225F30AB20B932CA5
:100930009E22442CEC0A20246B08F300ED2692251D
:10094000EB0A442CEC0A20246B08F300ED269225D8
:10095000442CE03E2022C4302B220800A2080319B8
:10096000CD2CB1080319B52C08006B08ED26EA0060
:100970002A3C0319C22C6A08793C0318C42C2A307B
:10098000EA00C52C6030EA00EA0A6A08F2006B0847
:10099000F300D6266A08A92408006B08ED26EA00B1
:1009A0002A3C0319DA2C6A08613C031CDC2C2A302F
:1009B000EA00DD2C7B30EA00EA036A08F2006B08EB
:1009C000C82C6B08F300ED26793C031DE92C6E3032
:1009D000EA2C7930EA00F2006B08F300D6266A08A8
:1009E000A9240800C608031D442DC60AB10803192E
:1009F000FD2CA2080319212D3C2C8711F408031D9E
:100A00005A28C7173E250230EE0094302B223708B3
:100A100045020319442DC5080319142DC5032830B8
:100A2000C302031CC4033E2D471C442DBC303702B7
:100A30000318442DBC30C5006030C3001D30C40015
:100A40003E2D8711F408031D5A283E250230EE0082
:100A500094302B22360837024502031D312DC7136F
:100A60000800BB30450203183B2DC50A2830C307D8
:100A70000318C40A3E2DC501C301C4014308202246
:100A80004408202240302B22080094302B22A3302F
:100A900084000008473C031D602D840A00084C3C7C
:100AA000031D602D840A00084C3C031D602D03309B
:100AB000F000A03020221E30202224302B22012AD8
:100AC000A33084000008563C031D792D840A0008D9
:100AD000543C031D792D840A0008473C031D792DE1
:100AE0000430F000F03020221E30202224302B224F
:100AF000012AA33084000008413C031D012A840A16
:100B00000008503C031D012A840A0008423C031DD2
:100B1000012A0530F000403020221F3020222430EE
:100B20002B22012AB400E03E2022C0302B223408C0
:100B30000800A030840000082C3C0319A72D0008F1
:100B40002A3C0319A72D00089225840A9B2D2030EA
:100B500092250800A030840000082E3C0319B42D13
:100B600000089225840AAC2D840A08004C30922596
:100B700041309225543092253A3092259925012A08
:100B80009925012A4C3092254F3092254E309225DE
:100B90003A3092259925012A9925012A5530922526
:100BA00054309225433092253A309225AA25012AC5
:100BB00054309225523092254B3092253A3092256E
:100BC0009925012A9925012A5330922550309225E2
:100BD000443092253A30922599254B309225743035
:100BE000922520309225922592259225012A58306F
:100BF000922554309225453092253A3092259925F8
:100C0000012A9925012A9925012A9925012A992540
:100C1000922592259225012A683020221F30202219
:100C200024302B22423092254F3092254430922599
:100C30003A3092259925012A9925012A4230922598
:100C400050309225443092253A3092259925012A38
:100C50009925012A48309225443092255330922517
:100C60003A3092259925012A992592259225922597
:100C7000012AF001A03084000008683C0319562EB8
:100C80000008703C0319592E0008733C03197A2E92
:100C900000086D3C03199A2E012AF300ED26031972
:100CA000552E72080F23F30A4E2E080000304D26F1
:100CB000012A31300F2332300F2333300F236130BC
:100CC0000F2363300F2366300F2367300F23683004
:100CD0000F2369300F236A300F236B300F236C30E2
:100CE0000F237A300F230D300F230A300F232630C5
:100CF0004D26012A840A0008743C031D012A840A37
:100D00000008313C0319922E0008323C03198F2E43
:100D10000008333C031D012A2830F300942E2730AD
:100D2000F300942E2630F300840A840A0008F200AF
:100D3000D626012A043084072930F3000008613CDC
:100D40000319D02EF30A0008633C0319D02EF30ACE
:100D50000008663C0319D02EF30A0008673C03190B
:100D6000D02EF30A0008683C0319D02EF30A0008BD
:100D7000693C0319D02EF30A00086A3C0319D02EEF
:100D8000F30A00086B3C0319D02EF30A00086C3CF0
:100D90000319D02EF30A00087A3C0319D02E012A39
:100DA000840A840A0008F200D626012A0317831653
:100DB0008C18D82E831273088D0072088C0083164D
:100DC0008C130C158B1355308D00AA308D008C14AC
:100DD0000C118B1783120313080003178312730877
:100DE0008D0083168C130C1483120C080313F2006D
:100DF00008000A158A140A14FF268A0108008207CF
:100E00000034003400340034003400340034003442
:100E100000340034003400340034003400340D3425
:100E200000340034003400340034003400347434AE
:100E30000034003400340A34003420347634003472
:100E400000340034003400340034003400346234A0
:100E50000034003400345F3400344C3478340034CF
:100E600000340034003442340034653446340034F5
:100E700000347534713400346B3400340034003481
:100E800000340034003400340034003400346F3453
:100E9000003400340034683400346E346D3400346F
:100EA0000034003400346C3400347234673400345D
:100EB0000034693470340034633400340034003456
:100EC0000034003400347A340034643400340034A4
:100ED0000034733479340034663400340034003420
:100EE00000346134773400346A3400340034003420
:100EF0004134003400340034003400340034003411
:100F00000034003400340034003400340034003441
:100F100000340034003400340034003400340D3424
:100F200000340034003400340034003400343534EC
:100F30000034003400340A34003420343D340034AA
:100F400000340034003400340034003400343F34C2
:100F50000034003400345F3400344C342F34003417
:100F60000034003400344234003433344634003426
:100F70000034373431340034283400340034003441
:100F80000034003400340034003400340034393488
:100F9000003400340034233400342C342E34003434
:100FA000003400340034293400343434263400341E
:100FB00000343834303400343A34003400340034EF
:100FC0000034003400342B34003424340034003432
:100FD00000345C34363400343F34003400340034A0
:100FE00000342D3432340034003400340034003402
:100FF0004134003400340034003400340034003410
:02400E00020F9F
:10420000730074006E003D005B0061002C002A000A
:104210005D000D000A006D00730067005F0078000C
:104220003D005B0079002C006E005D000D000A006F
:104230007000720069006E0074000D000A006800D2
:1042400065006C0070000D000A0000002A00680084
:104250006A00790079006E006E006E006E006E00DC
:104260006E006E006E000D000A0000005200650036
:104270007600200031002E0033000D000A000000FF
:00000001FF
